:02000000215786
:0300030002016691
:03000B0002016689
:0300130002016681
:03001B0002016679
:0300230002016671
:03002B0002016669
:0300330002030FB6
:03003B0002016659
:03004300020100B7
:03004B0002016649
:0300530002016641
:03005B000204BDDF
:0300630002016730
:03010000020C5A94
:030104000201ED08
:030108000202519F
:03010C0002027C70
:030110000202E404
:0101140032B8
:0101180032B4
:03011C000205FDDC
:03012000020000DA
:03012400020000D6
:0301280002043C92
:03012C0002046A60
:03013000020000CA
:03013400020000C6
:03013800020000C2
:03013C00020000BE
:03014000020000BA
:03014400020000B6
:03014800020000B2
:03014C00020000AE
:03015000020000AA
:03015400020000A6
:0A01570075817FE5826003020161FB
:0501610012076F21648C
:010166003266
:0E016700C0D0C086C082C083C0E0907F97E009
:0E0175004480F0907F69F0F0F0F0F0F0F0F0D0
:0E018300F0F0F0F0F0F0F0F0F0F0F0F0F0F04E
:0E019100F0F0F0F0F0F0F0F0F0F0907F97E07A
:03019F00557FF099
:0E01A200907F9AE030E423907F68F0F0F0F058
:0E01B000F0F0F0F0F0F0F0F0F0F0F0F0F0F021
:0E01BE00F0F0F0F0F0F0F0F0F0F0F0F0F0F013
:0E01CC00E5D8C2E3F5D8D0E0D083D082D0864B
:0301DA00D0D03250
:0801DD0075860090FFC37C054C
:0701E500A3E582458370F9D8
:0101EC0022F0
:0E01ED00C0E0C0F0C082C083C002C003C0D01A
:0E01FB0075D000C086758600E591C2E4F591CE
:0D020900908800E0F541907FAB7402F0900A
:090216007FAB7402F0E5326021B7
:04021F007A007B00E6
:0B022300C3EA9418EB64809480501232
:0E022E00907F69F0F0F0F0F0F0F0F00ABA0006
:02023C00010BB4
:02023E0080E35B
:02024000D08666
:0E024200D0D0D003D002D083D082D0F0D0E054
:01025000327B
:0E025100C0E0C0F0C082C083C0D075D000C035
:0E025F0086758600E591C2E4F591907FAB7440
:04026D0004F0D08643
:0B027100D0D0D083D082D0F0D0E0329B
:0E027C00C0E0C0F0C082C083C002C003C00456
:0E028A00C005C006C007C000C001C0D075D0BE
:0D02980000C086758600E591C2E4F59190E6
:0C02A5007FAB7408F0756E00756F0212DC
:0602B1001144757039755F
:0602B700710C75720212C9
:0C02BD001175907FD6E4F075D820D08633
:0E02C900D0D0D001D000D007D006D005D00490
:0D02D700D003D002D083D082D0F0D0E0322E
:0E02E400C0E0C0F0C082C083C0D075D000C0A2
:0E02F20086758600E591C2E4F591907FAB74AD
:0403000010F0D086A3
:0B030400D0D0D083D082D0F0D0E03207
:0E030F00C0E0C0F0C082C083C002C003C004C2
:0E031D00C005C006C007C000C001C0D075D02A
:0C032B0000C086758600756E00756F02BC
:0703370012114475704075BE
:06033E00710C7572021241
:0E0344001175907FD67402F0907FD67406F08B
:0503520075D810D086F3
:0E035700D0D0D001D000D007D006D005D00401
:0D036500D003D002D083D082D0F0D0E0329F
:0D037200907FA57480F0907FA6749AF01221
:0C037F00101B907FA6E542F012101B90AE
:0D038B007FA6E543F012101B907FA5744083
:01039800F074
:010399002241
:0D039A00907FA57480F0907FA6749AF012F9
:0C03A700101B907FA6E544F012101B9084
:0C03B3007FA6E545F012101B907FA6E528
:0B03BF0046F012101B907FA57440F068
:0103CA002210
:0A03CB0075440275450075460012E6
:0903D500039A75420375430012FE
:0203DE000372A8
:0103E00022FA
:0C03E100908800E536F09088007410252C
:0903ED0036F01201DD75420175C4
:0903F600431812037275440275EC
:0903FF00450075460012039A75D1
:08040800420375434412037224
:0104100022C9
:0E041100C0E0C0F0C082C083C0D075D000C073
:0E041F0086758600E591C2E4F591907FAA747F
:04042D0002F0D08683
:0B043100D0D0D083D082D0F0D0E032D9
:0E043C00C0E0C0F0C082C083C0D075D000C048
:0E044A0086758600E591C2E4F591907FA97455
:0704580004F0753001D086AD
:0B045F00D0D0D083D082D0F0D0E032AB
:0E046A00C0E0C0F0C082C083C0D075D000C01A
:0E04780086758600E591C2E4F591907FAA7426
:0704860004F0753101D0867E
:0B048D00D0D0D083D082D0F0D0E0327D
:0E049800C0E0C0F0C082C083C0D075D000C0EC
:0C04A60086758600E591C2E5F591D086D0
:0B04B200D0D0D083D082D0F0D0E03258
:0E04BD00C0E0C0F0C082C083C0D075D000C0C7
:0C04CB0086758600E591C2E7F591D086A9
:0B04D700D0D0D083D082D0F0D0E03233
:0C04E200907FEAE0FA8A20907F96E4F018
:0104EE0022EB
:0704EF00907FEAE0FA8A2188
:0104F60022E3
:0E04F700901713E0FA901715E0FB74802AFAB4
:0E05050074802BFBEA0303543FFCEAC423542A
:0E0513001FFA2CFAEB0303543FFCEBC42354F5
:0B0521001FFB2CFB90170AE0FC60029F
:02052C007A0053
:07052E0090170CE0FC6002D5
:020535007B0049
:0B053700EA2BFCC313F53A7544028B5D
:07054200458A4612039A7579
:090549006E08756F001211447573
:040552007047757108
:080556000C757202121175858B
:05055E003A731211A028
:010563002275
:0E056400907F96E0FA907F9674806502F0908A
:0E0572007FEBE0FA907FEAE0FB907FEFE0FC89
:0E0580003395E0FD8C057C00907FEEE0FE33AD
:0E058E0095E0FFEC2EFCED3FFD907FE9E0FED6
:05059C00BE0102800316
:0305A1000205F957
:0605A400BC0121BD001E98
:0E05AA00EAC40354F8FCEB25E0FD2C2400FC11
:0E05B800E43417FD907EC0E0FE8C828D83F04F
:0205C600803182
:0E05C800EAC40354F8FAEB25E0FB2AFA2400FB
:0E05D600FBE43417FC907EC0E0FD8B828C832A
:0E05E400F074012A2400FAE43417FB907EC163
:0705F200E0FC8A828B83F01C
:0305F90075380151
:0105FC0022DC
:0E05FD00C0E0C0F0C082C083C002C003C004D2
:0E060B00C005C006C007C000C001C0D075D039
:0D06190000C086758600E591C2E4F5919061
:0D0626007FAA7401F0120564753700D086BC
:0E063300D0D0D001D000D007D006D005D00422
:0D064100D003D002D083D082D0F0D0E032C0
:0E064E00907FEBE0FA907FEAE0FB907FEEE019
:0E065C00FC3395E0FD907F96E0FE907F967453
:0E066A00806506F0907F007401F0EAC403542E
:0E067800F8FEEB25E0FB2EFE2400FBE4341719
:0E068600FF8B828F83E0FB74012E2400FEE4C4
:0E0694003417FF8E828F83E0FE907FE9E0FF37
:0306A200BF810A0B
:0A06A500907F00EBF0907F01EEF073
:0806AF00907FE9E0FBBB821A19
:0306B700BA010C79
:0C06BA00907F00E4F0907F01E4F0800BE2
:0B06C600907F00E4F0907F0174B5F01D
:0806D100907FE9E0FBBB831BF5
:0306D900BA010D56
:0D06DC00907F007401F0907F01E4F0800B2E
:0B06E900907F00E4F0907F017412F09D
:0806F400907FE9E0FBBB841CD0
:0306FC00BA010D33
:0D06FF00907F007401F0907F01E4F0800C0A
:0C070C00907F007480F0907F017401F079
:05071800907FB5ECF03C
:01071D0022B9
:0C071E0075360D908800741DF0756B801E
:0A072A00756C3C1210E2756B8075CF
:090734006C0F1210E2756B807568
:09073D006C061210E2756B807568
:070746006C011210E27A00C1
:03074D00BAFF00F0
:02075000500A4D
:0A075200C0021201DDD0020A80F19E
:0A075C00756B80756C3C1210E2759D
:080766006B80756C0F1210E2AC
:01076E002268
:0E076F00907FA1E4F0907FAF7401F0907F9234
:0E077D007402F0758E3175892175880075C87B
:0E078B0000758D4075984075C04075870075EB
:0907990020007521007522007595
:0507A200230075470073
:0707A700C3E5479420501147
:0D07AE00E5472400F582E43417F583E4F0FC
:0407BB00054780E886
:0907BF00E4F540F53FE4F53CF5DA
:0707C8003BE4F53EF53D7531
:0B07CF003200753700753900907F93F1
:0E07DA00743CF0907F9C74FFF0907F967480CA
:0E07E800F0907F947470F0907F9D748FF0906D
:0E07F6007F97E4F0907F9574C2F0907F987426
:0E08040028F0907F9E7428F0907FF0E4F09032
:0E0812007FF1E4F0907FF2E4F0907FF3E4F0E9
:0E082000907FF4E4F0907FF5E4F0907FF6E432
:0E082E00F0907FF7E4F0907FF8E4F0907FF90F
:0E083C007438F0907FFA74A0F0907FFB74A0E7
:0E084A00F0907FFC74A0F0907FFD74A0F09001
:0E0858007FFE74A0F0907FFF74A0F0907FE010
:0E0866007403F0907FE17401F0907FDD7480E8
:0B087400F012124312071E7A007B00F6
:09087F00C3EA941EEB940050172B
:0C088800908800E0F54790880BE0F547F1
:09089400907F68F00ABA00010B24
:02089D0080E0F9
:0C089F001203E1907FD6E4F07A007B00A9
:0D08AB008A048B05C3EA94E0EB942E501AEA
:0E08B800C002C003C004C0051201DDD005D08F
:0A08C60004D003D0020ABA00010BAF
:0208D00080D9CD
:0D08D200907FD67402F0907FD67406F090EF
:0E08DF007FDE7405F0907FDF7405F0907FAC33
:0E08ED00E4F0907FAD7405F075A88075F810EA
:0D08FB00907FAE740BF0907FE27488F09057
:0C0908007FAB7408F075E81175320175C2
:0C0914003100753000C004C0051204F76B
:0A092000D005D004753400753501D0
:0D092A00907FAE7403F08C02BA00028003CF
:03093700020A3F72
:0C093A00853334907F9D748FF0907F9780
:0E0946007408F0907F9D7488F0907F9AE0FA1C
:0C09540074055AF533907F9D748FF0906D
:0D0960007F977402F0907F9D7482F0E53364
:0D096D0025E0FA907F9AE05405FB4AF5332F
:02097A00600C0F
:0C097C00907F96E0FA907F9674804AF01D
:0B098800756E00756F00C004C0051202
:0E0993001144D005D004901713E0FA74802AA6
:0609A100FAE533B404295D
:0309A700BAA000F3
:0209AA005024D7
:0D09AC00901713E004FB0B901713EBF09075
:0E09B9001713E0FB901715F0C002C004C00534
:0909C7001204F7D005D004D0029F
:0509D000E533B402262E
:0609D500C374049A5020D7
:0D09DB00901713E0FA1A1A901713EAF09023
:0D09E8001713E0FA901715F0C004C00512B7
:0609F50004F7D005D00458
:0509FB00E533B4081D06
:040A0000E534701950
:0A0A040074012535540FF5358535D2
:0C0A0E0075757600C004C0051213FED000
:030A1A0005D00400
:050A1D00E533B4011DEA
:040A2200E53470192E
:0A0A2600E53524FF540FF535853542
:0C0A300075757600C004C0051213FED0DE
:030A3C0005D004DE
:0E0A3F00C004C0051201DDD005D004907F96E2
:0E0A4D00E0FA907F96747F5AF0907F977408BD
:0A0A5B00F0C3EC9400ED9402400893
:080A6500907F96E0FA20E608FC
:080A6D00C3E49C74089D5013C2
:0E0A7500907F96E0FA907F9674406502F07CC8
:050A8300007D0080056C
:050A88000CBC00010D93
:050A8D00E538B4010E84
:0D0A9200C004C0051204F7D005D00475386B
:010A9F000056
:070AA000E531700302092A91
:0A0AA700907FC9E0FA7003020C2DE5
:0E0AB100907F96E0FA907F9674806502F09038
:090ABF007DC0E0FABA2C028003AC
:030AC800020B36E8
:050ACB007532007B0004
:030AD000BB640004
:020AD300501CB5
:0E0AD500C002C003C004C0051201DDD005D070
:0D0AE30004D003D00290880FE0F5470B808F
:010AF000DF26
:0D0AF100C002C004C00512071E1203E1126E
:0C0AFE0004F7D005D004D002756E00751E
:0D0B0A006F01C002C004C005121144D005E7
:090B1700D004D00275704D757117
:0B0B20000C757202C002C004C0051278
:0B0B2B001175D005D004D002020C2D83
:030B3600BA2A3B9D
:0D0B3900907F987420F0C002C004C0051227
:0E0B460001DDD005D004D002907F987428F015
:020B54007B0024
:030B5600BB0A00D7
:050B59004003020C2D19
:0E0B5E00C002C003C004C0051201DDD005D0E6
:080B6C0004D003D0020B80E26B
:030B7400BA2B1A7F
:080B7700907FC9E0FBBB4012B6
:0E0B7F00C002C004C005121205D005D004D07B
:040B8D0002020C2D27
:030B9100BA101F78
:0E0B9400907F96E0FB907F9674806503F0C022
:0E0BA20002C004C00512103DD005D004D002E0
:030BB000020C2D07
:030BB300BA111262
:0E0BB600C002C004C00512106AD005D004D0E1
:040BC40002020C2DF0
:030BC800BA12124C
:0E0BCB00C002C004C00512108FD005D004D0A7
:040BD90002020C2DDB
:030BDD00BA130B3D
:0B0BE000907DC1E0FB908800F0804297
:030BEB00BA141128
:0E0BEE00C002C004C0051211DDD005D004D035
:030BFC0002802E46
:030BFF00BA151D07
:0C0C0200907DC1E0F575907DC2E0F576B4
:0E0C0E00C002C004C0051213FED005D004D0F1
:030C1C0002800E45
:030C1F00BA160BF7
:0B0C2200C004C0051213A3D005D004CD
:0B0C2D00907FC9E4F075310002092A35
:010C38002299
:070C3900535550454E4400E5
:070C4000524553554D4500DC
:060C470020566F6C200036
:0D0C4D004441425553422076312E30300094
:0E0C5A00C0E0C0F0C082C083C002C003C0046E
:0E0C6800C005C006C007C000C001C0D075D0D6
:0D0C760000C086758600E591C2E4F59190FE
:0E0C83007FAB7401F0907FE8E0FA907FE9E02B
:060C9100FBBB0002800322
:030C9700020D3813
:030C9A00BA801409
:0E0C9D00907F007401F0907F01E4F0907FB52D
:060CAB007402F0020ECD00
:050CB100BA820280037D
:030CB600020D1D0F
:080CB900907FECE0FCBC01009F
:020CC1004021D0
:060CC300C374079C401BF6
:0E0CC900EC24FF25E0FD24C6F582E4347FF51F
:0D0CD70083E0FD530501907F00EDF0802BC0
:030CE400BC8100D0
:020CE7004021AA
:060CE900C374879C401B50
:0E0CEF00EC247F25E0FC24B6F582E4347FF58A
:0D0CFD0083E0FC530401907F00ECF08005C3
:050D0A00907F00E4F001
:0E0D0F00907F01E4F0907FB57402F0020ECDEB
:050D1D00BA8102800311
:030D2200020EC5F9
:0E0D2500907F00E4F0907F01E4F0907FB574C1
:050D330002F0020ECDEC
:030D3800BB012DCF
:060D3B00BA0003020ECD18
:030D4100BA0211E2
:0D0D4400755900C002C003120EF0D003D09C
:040D510002020ECDBF
:050D5500BA2102800339
:030D5A00020ECDB9
:0B0D5D00753701907FC5E4F0020ECD59
:030D6800BB031FAB
:060D6B00BA0003020ECDE8
:050D7100BA020280033C
:030D7600020ECD9D
:0D0D7900755901C002C003120EF0D003D066
:040D860002020ECD8A
:030D8A00BB065451
:050D8D00BA80028003A2
:030D9200020EC589
:080D9500907FEBE0FCBC0115AE
:0C0D9D007CFB7D0F8D067F00907FD4EE64
:090DA900F0907FD5ECF0020ECDB4
:0A0DB200907FEBE0FCBC020280031E
:030DBC00020EC55F
:0A0DBF00907FEAE0FCBC0002800314
:030DC900020EC552
:0C0DCC007C3B7D0F8D067F00907FD4EEF5
:090DD800F0907FD5ECF0020ECD85
:060DE100BB0703020EC572
:030DE700BB081036
:0D0DEA00AC48907F00ECF0907FB57401F0F4
:030DF700020ECD1C
:030DFA00BB093101
:050DFD00BA00028003B2
:030E0200020EC518
:0E0E0500907FEAE0FCC374019C5003020EC50E
:080E1300907FEAE0FCBC000A3C
:0A0E1B00901721E4F0901722E4F094
:090E2500907FEAE0F548020ECDD1
:030E2E00BB0A27D5
:050E3100BA81028003FC
:030E3600020EC5E4
:0E0E3900907FECE0FA2420FAE43417FC8A8261
:0E0E47008C83E0FA907F00F0907FB57401F08C
:030E5500020ECDBD
:050E5800BB0B0280034A
:030E5D00020EA9D9
:0D0E6000901720E4F0907FECE0FABA011A40
:080E6D00907FEDE0FABA0012DB
:0E0E7500907FEAE0FA901721F0C0031204E229
:040E8300D0038046D2
:080E8700907FECE0FABA023E94
:080E8F00907FEDE0FABA003695
:0D0E9700C0031204EFD003907FEAE0FA9050
:050EA4001722F080247C
:050EA900BB12028017DE
:050EAE00BB8102800D74
:050EB300BB8302800872
:050EB800BB8202800373
:030EBD00BB8405EE
:050EC00012064E80083F
:080EC500907FB47403F0800675
:060ECD00907FB47402F0F6
:020ED300D086C7
:0E0ED500D0D0D001D000D007D006D005D00478
:0D0EE300D003D002D083D082D0F0D0E03216
:0B0EF000907FECE0F55AC39401401D18
:070EFB00C37407955A40166D
:0D0F0200E55A24FF25E0FA24C6F582E43408
:090F0F007FF583AA59EAF0802263
:070F1800C3E55A9481401B60
:070F1F00C37487955A4014CA
:0D0F2600E55A24FF25E0FA24B6F582E434F4
:070F33007FF583AA59EAF0E3
:010F3A002294
:0E0F3B000902BA000301004000090400000092
:0E0F49000101000009240100013D0001010C1E
:0E0F570024020110070002030000000D240612
:0E0F650003010215000300030000092403022B
:0E0F7300010100010009240304020300030031
:0E0F8100092403050306000100090401000015
:0E0F8F00010200000904010101010200000737
:0E0F9D002401020101000B24020102021001D6
:0E0FAB0080BB00090588050001010000072534
:0E0FB900010000000009040200020000000018
:0E0FC7000705820240000007050202400000FC
:0E0FD50009040201030000000007058202402B
:0E0FE30000000705020240000009058905A074
:0A0FF1000101000000FFFFFFFF00F8
:0E0FFB00120100010000004047059999000115
:0E10090000000001000000000000000902BA13
:0410170000030100D1
:02101B007A0059
:03101D00BA050011
:02102000501767
:08102200907FA5E0FB30E00522
:05102A00900001800DA3
:0A102F00C0021201DDD0020A80E4C5
:0310390090000123
:01103C002291
:0E103D00907DC1E0F9A3E0FAA3E0FB7C007D0A
:04104B007EEB6012C6
:0E104F0089828A83E0A3A982AA838C828D8382
:04105D00F00CDBEECA
:08106100907DC3E0907FB9F01F
:011069002264
:0E106A00907DC1E0F9A3E0FAA3E0FB7CC47D19
:041078007DEB60E5C7
:0E107C008C828D83E00C89828A83F0A3A98286
:04108A00AA83DBEE6C
:01108E00223F
:0E108F00907FA57480F00586907DC1E00586F7
:0E109D00A3F012101B907FA60586A3A3E0F916
:0510AB006016A305869C
:0D10B000907FA60586E0A30586F0C0011222
:0610BD00101BD001D9ED6B
:0610C300907FA57440F0CF
:0110C9002204
:0810CA009088027401F07A0025
:0310D200BAFF0062
:0210D500500ABF
:0A10D700C0021201DDD0020A80F110
:0110E10022EC
:0510E200E56BB4C0083D
:0810E700908803E56CF080061F
:0610EF00908802E56CF0A0
:0410F5007A007B0002
:0B10F900C3EA9432EB6480948050073F
:051104000ABA00010B16
:0211090080EE76
:01110B0022C1
:0A110C00908803E56DF005397A00C4
:03111600BA2800F4
:02111900500381
:03111B000A80F84F
:05111E00E539B41008E2
:0811230090880274C0F0800EF8
:05112B00E539B42009C4
:091130009088027480F07539000A
:021139007A003A
:03113B00BA2800CF
:02113E0050035C
:031140000A80F82A
:011143002289
:04114400E56F6002F1
:0211480080071E
:07114A007A007539008005F1
:051151007A4075391021
:09115600E56E2AFAE56E2539F573
:0A115F003990880274802AF07A00AB
:08116900C3EA648094A850035E
:031171000A80F5FC
:011174002258
:06117500AA70AB71AC7220
:0C117B008A828B838CF01214EEFD601849
:0D1187008D6DC002C003C00412110CD00415
:09119400D003D0020ABA00010BDD
:02119D0080DCF4
:01119F00222D
:0D11A000E573C4540FFA53020FC374099A8B
:0211AD005006EA
:0611AF0074372AFB8004E6
:0411B50074302AFB6D
:0C11B9008B6DC00312110CD003AA7353FD
:0811C500020FC374099A5006E1
:0611CD0074372AFB8004C8
:0411D30074302AFB4F
:0511D7008B6D12110CEC
:0111DC0022F0
:0711DD00907DC3E0FA600FF2
:0C11E400907DC1E0F56E907DC2E0F56FDB
:0311F00012114495
:0C11F300907DFFE4F07570C475717D758F
:0511FF007201121175E0
:0112040022C7
:021205007A0469
:03120700BA4000EA
:02120A0050365C
:0E120C00EA24C0F582E4347DF583E0FB7C002B
:03121A00BC08000D
:02121D0050205F
:06121F008B05ED30E70B2A
:0B122500907F967442F074C3F08008C4
:08123000907F96E4F07481F058
:07123800EB25E0FB0C80DB5D
:03123F000A80C55D
:011242002289
:041243007A007BEFC3
:03124700BA1000DA
:02124A00502032
:0E124C0074112BFB2400FCE43418FD8C828D01
:0E125A0083E4F0EA2400F582E43419F583E41D
:04126800F00A80DB2D
:01126C00225F
:0E126D0074F82400F58274033484F583E4F0F1
:0E127B0074F92400F58274033484F583E4F0E2
:0E12890074FA2400F58274033484F583E4F0D3
:0E12970074FB2400F58274033484F583E4F0C4
:0E12A50074FF2400F58274033484F583E4F0B2
:0112B3002218
:0E12B4001203CB12126D7AC07B877C0174018D
:0E12C2002AFDE43BFE8C078A828B838CF0743D
:0E12D000011214BF2DFAE43EFB8F048D828EB6
:0E12DE00838FF074061214BF74012AFDE43BE6
:0E12EC00FE8C078A828B838CF0E41214BF7490
:0E12FA00012DFAE43EFB8F048D828E838FF06F
:0E130800740B1214BF74012AFDE43BFE8C0727
:0E1316008A828B838CF074081214BF74012D30
:0E132400FAE43EFB8F048D828E838FF07401FD
:0E1332001214BF2AFDE43BFE8C078A828B83D7
:0E1340008CF0E41214BF74012DFAE43EFB8F12
:0E134E00048D828E838FF074031214BF7D0015
:03135C00BD0600CB
:02135F0050122A
:0B1361008A828B838CF00ABA00010B1B
:07136C00E41214BF0D80E93B
:0D1373008A828B838CF0E5741214BF74F92C
:0E1380002400F58274033484F583740FF07436
:0E138E00FE2400F58274033484F5837401F0AC
:06139C001203E11204F748
:0113A2002228
:0D13A300907DC1E0FA2400FBE43419FC90B9
:0E13B0007DC2E0FD8B828C83F075F011EAA403
:0313BE00FA7B00B7
:0313C100BB10005E
:0213C4005024B3
:0E13C600EA2400FCE43418FDEB2CFCE43DFDB1
:0E13D40074042B24C0F582E4347DF583E0FE22
:0813E2008C828D83F00B80D793
:0E13EA00EA2400FAE43418FB74102AF582E4B9
:0513F8003BF583E4F069
:0113FD0022CD
:0413FE00E57660022E
:02140200801652
:0C140400740F5575FA8A752400F582E417
:0A1410003419F583E0F5741212B4EC
:0A141A001210CA756E00756F001203
:0614240011447570B9755A
:06142A007114757202123C
:0B1430001175E576B402047401800120
:01143B00E4CC
:03143C00FA700F34
:0C143F0074012575F573C0021211A0D0D5
:03144B0002800A12
:0A144E00857573C0021211A0D002D0
:0C145800756E00756F01C002121144D0C7
:0414640002EA701A0E
:0D14680075F011E575A4FA2400FAE43418BB
:09147500FB8A708B717572011283
:04147E00117580362E
:021482007A00EE
:03148400BA10009B
:02148700502FE4
:0D148900EA2400F582E43419F583E0FBE568
:0414960075B5031B0A
:0E149A0075F011EAA4FB2400FBE43418FC8B6F
:0914A800708C71757201C0021212
:0414B1001175D002DF
:0314B5000A80CCDE
:0114B8002211
:0614B90050726F67200075
:0E14BF00C8C0E0C8C0E0E5F0600B14600F1478
:0714CD00601114601280158C
:0714D400D0E0A882F6800EB3
:0514DB00D0E0F08009E3
:0414E000D0E08005D3
:0514E400D0E0A882F237
:0414E900C8D0E0C8BF
:0114ED0022DC
:0E14EE00C8C0E0E5F0600D14600F14600F142C
:0614FC00601074FF800F78
:05150200A882E6800A4A
:03150700E080077A
:04150A00E4938003E3
:03150E00A882E2CE
:04151100F8D0E0C866
:0115150022B3
:00000001FF
